:020000000329D2
:08000800FF00030E8312031335
:10001000B4000A0EB500040EB6008A110A122B298C
:1000200000000000CC0B102808004A08CE00CD01CB
:100030000310CE0DCD0DCE0DCD0DCE070318CD0A7C
:10004000CE070318CD0A2E30CE070318CD0A003094
:100050004D078A004B08CD004E08820000308A0010
:100060000030CE004A30432800308A000030CE00F5
:100070005630432800308A000030CE0059304328E3
:100080000030CE005D30CD070318CE0A4E088A003E
:100090004D0882000134043407340A340234053434
:1000A000083400340334063409340B340434023485
:1000B000013408341034203440343134343437348B
:1000C0002A343234353438343034333436343934F5
:1000D0002334C308031D6D280800F9300000000018
:1000E0000000000000000000000000000000000010
:1000F000000000000000000000000000FF3E031DA3
:100100006E28000000000000000000000000000059
:1001100000000000000000000000000000000000DF
:1001200000000000C30B6D28080083169816831288
:100130000C1E97284308990008000330831203130C
:10014000C3000130C4000230C500783083160604B5
:100150008600F830060586008312C6010330460289
:100160000318D2284408CA004608CB001520860090
:100170000A30CC008A110A1210200608C800C701F4
:10018000043047020318D0284508CA004708CB00AE
:10019000152048058A110A12031DD528C70AC02850
:1001A000C60AAE28FF30CC0008004308CA00460843
:1001B000CB00C901CB0DC90DCB0DC90DFC30CB0552
:1001C0004708CB071520CC0008000730831603131F
:1001D0009F0004309800813099008312980198178D
:1001E000C030831681009D204C08C200420A8A114B
:1001F0000A120319F3284208C300C4019520FA30FB
:10020000C3006920F328D53083120313A000C43043
:10021000A100BB30A200DC30A300A401A501A6010F
:10022000A701A801A901AA01AB01AC01AD01AE0172
:10023000AF01BC01BD01B701B801BE01BF01C001E2
:10024000C101B001B101B201B301BA01BB01B901F1
:100250008A110A12E52883120313360E8400350E24
:0C0260008A00340E8300FF0E7F0E0900A0
:02400E003A3F37
:00000001FF
